:1000000000308A0092280000851283168512831220
:10001000851005118316851005111F169F121F17D5
:1000200083129F171F141F1383161F149F101F1175
:100030009F1100308312C1001F08E33941049F0063
:100040009F28483084000008031934280130C1007B
:10005000C001C00B2928C10B28284A30C000C00BA2
:100060002F283228800B262808009F1449109F1C37
:10007000491449183F2849109F1C491439289F18D2
:100080003F281E08C30083161E088312CA001E08DC
:10009000CB004A08C1004B08C200080035204208C6
:1000A000C8004108C70035204108C70742080318A7
:1000B000420FC80735204208C3004108C70742085D
:1000C0000318420FC80735204108C7074208031824
:1000D000420FC807480CC300470CC200C30CC20C37
:1000E0003F30C3054208C1004308C200A3284808A6
:1000F000C30047080319C803C703430403198F2823
:10010000851405112730C000C00B842887280515E9
:1001100085102730C000C00B8B288E2877288510CB
:100120000511C72884011F3083051F1383161F1074
:100130009F101F119F1183129A019C0104286430A3
:10014000C80021204E284208C6004108C5004608C4
:10015000013C0318B428FF3A031DB2284508C93CE6
:100160000318B4288512CF284608013C0318C1287B
:10017000FF3A031DBF2845088B3C0318C12885168C
:10018000CF2885160330C8002030C7007728851295
:100190000230C7009630C8002120C70BCA28A22809
:0201A0006300FA
:02400E00443F2D
:00000001FF
